:100000000C9434000C9451000C9451000C94510049
:100010000C9451000C9451000C9451000C9451001C
:100020000C9451000C9451000C9451000C9451000C
:100030000C9451000C9451000C9451000C945100FC
:100040000C9451000C9451000C94100B0C94510022
:100050000C94420B0C9451000C9451000C945100E0
:100060000C9451000C94510011241FBECFEFD8E026
:10007000DEBFCDBF13E0A0E0B1E0E2E5FDE102C0EC
:1000800005900D92A234B107D9F723E0A2E4B3E0C2
:1000900001C01D92A639B207E1F70E9426070C9411
:1000A000A70E0C940000FC0181E0808372836183C1
:1000B000709344036093430384E1838314828FEF3E
:1000C0009FEF9683858390878783928781871486A5
:1000D0001386168615860895FC0183E08083808947
:1000E000887F808B81E0878713820895FC0180815F
:1000F000823089F485E080834134510578F4828927
:10010000887F828B118A748B638B568B458B13820D
:1001100080E090E008958CEF9FEF08958FEF9FEFC0
:100120000895CF92DF92EF92FF920F931F93CF9398
:10013000DF9300D0CDB7DEB77C016B015A834983D2
:10014000FC0180818530D1F44589568963897489A1
:100150008E010F5F1F4F9601C70141960E94480311
:10016000992364F49F938F9380E091E09F938F9302
:100170000E94990B0F900F900F900F90F7018081C4
:100180008330D1F48E010F5F1F4F960140E050E0A5
:1001900060E070E0C7010F960E944803992364F461
:1001A0009F938F9380E091E09F938F930E94990B90
:1001B0000F900F900F900F90F70180818430D1F451
:1001C0008E010F5F1F4F960140E050E060E070E04D
:1001D000C70147960E944803992364F49F938F9325
:1001E00080E091E09F938F930E94990B0F900F9066
:1001F0000F900F9080E090E00F900F90DF91CF91E3
:100200001F910F91FF90EF90DF90CF9008952F9264
:100210003F924F925F926F927F928F929F92AF9296
:10022000BF92CF92DF92EF92FF920F931F93CF93E3
:10023000DF9300D000D0CDB7DEB75C015C834B8389
:10024000222E332E38018DB69EB6C42ED52E8DB7F4
:100250009EB78C199D090FB6F8949EBF0FBE8DBF37
:10026000EDB7FEB731962F01CE0103967C018F01C9
:100270009601AB01BE016F5F7F4FC50104960E94DE
:10028000220299230CF448C08A81877090E0F5011E
:10029000238130E08217930751F084E08083808DC2
:1002A000887F808F82E0878B8AEF9FEF35C08981BE
:1002B000813049F018F08230D9F025C0F2E0CF1A31
:1002C000D10829F40EC082E0F50180831CC0F20140
:1002D000A22DB32D4C0C5D1C81918D93E415F50579
:1002E000D9F7F301D182C08286E0F50180830BC08B
:1002F00084E0F5018083808D887F808F82E0878B0A
:100300008AEF9FEF09C08091430390914403F50168
:100310009283818380E090E00FB6F8949EBE0FBE7A
:100320008DBE0F900F900F900F90DF91CF911F9186
:100330000F91FF90EF90DF90CF90BF90AF909F9084
:100340008F907F906F905F904F903F902F90089587
:10035000FC0121813281261B370B32832183121647
:1003600013061CF480E090E008958BEF9FEF089552
:10037000FC01E627FF27EE0FFF1FEA5EFE4F892FE5
:10038000992720813181822793270895FA0193E8E4
:10039000980F923070F420813181A9014F5F5F4F37
:1003A00051834083DB01A20FB31F9DE79C9390E232
:1003B000892720813181A9014F5F5F4F518340839D
:1003C000FB01E20FF31F80830895982F80FF0BC07D
:1003D00086958695837011F082E001C081E0929548
:1003E0009695977003C09695977080E097700895E2
:1003F000FC019081913049F018F0923061F011C009
:1004000081818770880F8061089581818295880F2E
:10041000807E8160089581818295880F807E8960C9
:10042000089580E00895FC018FEF9FEF9283818310
:100430009683858394838383128611861086178220
:10044000108208953F924F925F926F927F928F92A7
:100450009F92AF92BF92CF92DF92EF92FF920F9353
:100460001F93CF93DF9300D000D0CDB7DEB70097B6
:1004700009F4EAC06115710509F4E9C04115510597
:1004800009F4E8C00115110509F4E7C0E114F1040D
:1004900009F4E6C0380149017A8369839C838B8320
:1004A0002115310509F499C08A01C12CD12C689419
:1004B000442445F833243394590121E0A21AB108A9
:1004C000AB81BC8113968D919C91149799239CF4D8
:1004D000F80180818E3709F070C0CA14DB0420F463
:1004E00081818E3709F470C0EB81FC818781908512
:1004F0009483838362C0F80150802EE7521219C0A2
:10050000CA14DB0420F421812E3709F45DC0AB81CD
:10051000BC8117962D913C911897AC014F5F5F4FAE
:100520004217530709F450C016963C932E93159723
:100530005DC0BDE75B1204C0EB81FC8130823DC031
:10054000AB81BC818C91882319F01C92508054247B
:10055000652DEB81FC81818192810E94B801AB8184
:10056000BC8112969C938E93119717962D913C9176
:10057000189713968D919C91149702962817390716
:1005800041F4852D0E94E501E981FA819183808300
:1005900014C0821793078CF4AB81BC8119968D919E
:1005A0009C911A979C012F5F3F4F1A963C932E9374
:1005B0001997F301E80FF91F5082EB81FC818781C5
:1005C0009085019690878783FFEFCF1ADF0A0F5F30
:1005D0001F4F8C149D0409F073CFAB81BC8113961F
:1005E0008D919C91149799233CF06401EB81FC81DF
:1005F00025813681332334F4D7011D921C928EE07D
:1006000092ED30C00496281739073CF0EB81FC814D
:1006100081819281883B904F31F0D701CD92DC925D
:100620000EE012ED0AC0EB81FC8181859285029774
:10063000D7018D939C930C2D1D2D8B819C810E9445
:100640001302802F912F0EC08EE092ED0BC08EE032
:1006500092ED08C08EE092ED05C08EE092ED02C0F2
:100660008EE092ED0F900F900F900F90DF91CF9151
:100670001F910F91FF90EF90DF90CF90BF90AF90C0
:100680009F908F907F906F905F904F903F900895D4
:100690005F926F927F928F929F92AF92BF92CF9212
:1006A000DF92EF92FF920F931F93CF93DF9300D0CF
:1006B000CDB7DEB7009709F473C06115710521F459
:1006C0004115510509F06FC02115310509F46EC0BF
:1006D0000115110509F46DC0380179015A014B016A
:1006E0008C0181E090E09A8389838EE7F901808311
:1006F0006FEF8FEF9FEF0E94B8016C01AE014F5F6B
:100700005F4FB7018FEF0E94C601C8010E94F80138
:10071000582E682FC6010E94B8016C01AE014F5FD0
:100720005F4FB701852D0E94C601F80180818111BC
:1007300019C0A114B104B1F084018A0C9B1C5801AA
:10074000F80161918F01C6010E94B8016C01AE01F0
:100750004F5F5F4FB701F50180810E94C60180168F
:10076000910669F7C094D094AE014F5F5F4FB70117
:100770008C2D0E94C601AE014F5F5F4FB7018D2DDA
:100780000E94C60189819A81F701E80FF91F2EE7BF
:1007900020830196F3019183808380E090E00BC079
:1007A0008EE092ED08C08EE092ED05C08EE092EDF5
:1007B00002C08EE092ED0F900F90DF91CF911F91CC
:1007C0000F91FF90EF90DF90CF90BF90AF909F90F0
:1007D0008F907F906F905F900895CF93882331F032
:1007E0008091420381608093420305C0809142035F
:1007F0008E7F809342038091420382608093420304
:100800006091420380E00E94950662E080E00E94D1
:10081000D60600C064E080E00E948106C82F62E036
:1008200080E00E94DA0600C062E080E00E94D60606
:1008300000C064E080E00E948106C295C07F8F7096
:10084000C82B62E080E00E94DA068C2FCF910895D9
:1008500080E00E94ED038823DCF300C080E00E946A
:10086000ED03089562E080E00E94D60600C062E0D9
:1008700080E00E94DA060895CF93C82F662331F0F6
:100880008091420381608093420305C080914203BE
:100890008E7F80934203809142038D7F8093420339
:1008A0006091420380E00E949506809142038F7719
:1008B00080934203809142038F7B80934203809117
:1008C00042038F7D80934203809142038F7E809309
:1008D0004203CC232CF4809142038068809342032E
:1008E000C6FF05C080914203806480934203C5FF28
:1008F00005C080914203806280934203C4FF05C01B
:10090000809142038061809342036091420380E0C2
:100910000E9495060E943204809142038F77809353
:100920004203809142038F7B809342038091420374
:100930008F7D80934203809142038F7E8093420398
:10094000C3FF05C080914203806880934203C2FFC9
:1009500005C080914203806480934203C1FF05C0BB
:1009600080914203806280934203C0FF05C0809162
:1009700042038061809342036091420380E00E94C1
:1009800095060E9432048091420380618093420365
:10099000809142038062809342038091420380648D
:1009A0008093420380914203806880934203609168
:1009B000420380E00E949506CF910895CF93C82FFF
:1009C0000E94280460E08C2F0E943C04CF9108957F
:1009D000611104C080580E94DE04089580540E9472
:1009E000DE04089581E00E94DE040895882331F03A
:1009F00080914203877F8093420305C08091420328
:100A00008860809342036091420380E00E949506D3
:100A1000089582E00E94DE040895CF93C82F0E94BB
:100A20002804CA3049F4803410F080E001C080E42A
:100A300080580E94DE0413C0803129F460E080EC0D
:100A40000E943C0406C0803521F460E080E80E94EA
:100A50003C040E94280461E08C2F0E943C04CF914A
:100A60000895CF93DF93EC012196FC0180818823C8
:100A700029F00E940D0589918111FBCFDF91CF9163
:100A800008951F93CF93DF93182F0E94780610923A
:100A900042036091420380E00E94950680EA9FE055
:100AA0000197F1F780914203806280934203809125
:100AB00042038061809342036091420380E00E9480
:100AC00095060E94320480EE94E00197F1F70E94AF
:100AD0003204C0E1D0E0CE010197F1F70E94320468
:100AE000CE010197F1F7809142038F7E80934203FC
:100AF0006091420380E00E9495060E943204219793
:100B0000F1F788E20E94DE0488E00E94DE040E9481
:100B1000F20486E00E94DE04812F0E94DE04DF9151
:100B2000CF911F9108958DE00E9441050E94090513
:100B300080E00E94F6040895CF92DF92EF92FF9238
:100B40000F931F93CF93DF938C017B01C901F801B1
:100B500001900020E9F73197BF01601B710B0E94E3
:100B6000760B670120E1C20ED11CE7019C012E1912
:100B70003F09F80101900020E9F73197BF01601BA0
:100B8000710BC9018C0F9D1F0E94760BF801E80FB5
:100B9000F91F80818993CC15DD0559F7F701108A7B
:100BA000DF91CF911F910F91FF90EF90DF90CF9049
:100BB0000895AF92BF92CF92DF92EF92FF920F9380
:100BC0001F931F930F93FF92EF925F934F933F9367
:100BD0002F939F938F937F936F9386E193E09F93DF
:100BE0008F93BF92AF92DF92CF920E94AF0B8DB7DF
:100BF0009EB742960FB6F8949EBF0FBE8DBF1F9151
:100C00000F91FF90EF90DF90CF90BF90AF9008953D
:100C10006F927F92AF92BF92CF92DF92EF92FF924C
:100C20000F931F93CF93DF93CDB7DEB7C254D10993
:100C30000FB6F894DEBF0FBECDBF3C012091490333
:100C400030914A0341E150E0BE016F5F7F4F0E9447
:100C50009C05F301E85BFF4FE080F1800281138186
:100C60003497208131814281538134976081718131
:100C7000828193810F2EF1E1AF2EB12CF02DFE0178
:100C800072966F010E94D90540E150E0BE016F5F8E
:100C90007F4FCE0183960E948A0B40E150E0B6015F
:100CA000CE01C3960E948A0B60E080E00E94E804B7
:100CB000CE0183960E94310561E080E00E94E80445
:100CC000CE01C3960E943105CE5BDF4F0FB6F8947C
:100CD000DEBF0FBECDBFDF91CF911F910F91FF906F
:100CE000EF90DF90CF90BF90AF907F906F9008957E
:100CF0000E94DE0683E08A95F1F7000010924B0314
:100D0000089581110EC0683070F480914B03082E55
:100D1000000C990B02C0959587956A95E2F7817052
:100D200008958FEF08958FEF0895CF9381110DC02F
:100D3000C62F60934B038EE40E94E4068C2F0E9422
:100D400014070E940B0780E001C08FEFCF91089538
:100D5000CF93DF93811124C0683020F580914B033D
:100D6000442349F0C1E0D0E002C0CC0FDD1F6A95FA
:100D7000E2F7C82B09C0C1E0D0E002C0CC0FDD1FF4
:100D80006A95E2F7C095C823C0934B038EE40E9496
:100D9000E4068C2F0E9414070E940B0780E003C01A
:100DA0008FEF01C08FEFDF91CF91089541E00E9456
:100DB000A806089540E00E94A80608951092B90080
:100DC0008DEF8093B800089594EA9093BC00ECEB0B
:100DD000F0E090819923ECF79091B900987F9830DA
:100DE00011F09031A1F48093BB0084E88093BC00A3
:100DF000ECEBF0E080818823ECF79091B900987FCC
:100E0000983139F081E0903429F480E0089581E050
:100E1000089580E0089584E98093BC00ECEBF0E055
:100E2000808184FDFDCF08958093BB0084E880938A
:100E3000BC00ECEBF0E080818823ECF79091B900E6
:100E4000987F81E0983209F480E008954F925F9294
:100E50006F927F928F929F92AF92BF92CF92DF92CA
:100E6000EF92FF920F931F93CF93DF93CDB7DEB72F
:100E7000C350D2400FB6F894DEBF0FBECDBF0E9464
:100E800093050E949E0A68EC70E0CE0101960E94D4
:100E90005300CE0101960E946C004AE050E0BE0172
:100EA000665E7F4FCE0101960E9491006AE070E07D
:100EB000CE014A960E94AA0A64E170E0CE018051F8
:100EC0009E4F0E94CE0A61E070E0CE0101960E9422
:100ED000A801059681F44AE050E0BE01665E7F4FAE
:100EE000CE0101960E9491006AE070E0CE014A9620
:100EF0000E94AA0AE1CF00E010E020E030E044E1E7
:100F000050E0BE0160517E4FCE0101960E94070164
:100F10008C019923ACF40A3F8FEF1807B1F444E138
:100F200050E0BE01605A7E4FCE0101960E949100B2
:100F300064E170E0CE01805A9E4F0E94AA0A05C06B
:100F40008981823009F0B8CF03C0802F912FFEC075
:100F500084EA90E7ADE9BFE38CA39DA3AEA3BFA352
:100F60008DEC9CECA0EBB1E488A799A7AAA7BBA73E
:100F700080E090E0A8ECB2E48CA79DA7AEA7BFA745
:100F800083E090E099AB88AB85E293E09BAB8AABC2
:100F900082E090E09DAB8CAB2E01E6E74E0E511C3B
:100FA0005F924F923E01F6E36F0E711C7F926F923B
:100FB0008CA09DA0AEA0BFA0C8A4D9A4EAA4FBA405
:100FC0000CA51DA52EA53FA548A959A96AA97BA9CD
:100FD0008CA99DA90E945C09F20140815181B30155
:100FE000CE0101960E94760048E450E0BE016858A8
:100FF0007F4FCE0101960E94910068E470E0CE011F
:1010000088589F4F0E94AA0A0F900F900F900F9040
:1010100060E970E0CE01805A9E4F0E94CE0A61E0E6
:1010200070E0CE0101960E94A801059689F448E47B
:1010300050E0BE0168587F4FCE0101960E9491009A
:1010400068E470E0CE0188589F4F0E94AA0AE0CF62
:101050008E0113959E0120543F4F40E950E0BE01A0
:10106000605A7E4FCE0101960E9407018C019923A0
:101070009CF40696B1F444E150E0BE0160517E4F0D
:10108000CE0101960E94910064E170E0CE01805192
:101090009E4F0E94AA0A05C08981863009F0B8CF08
:1010A00003C0802F912F52C0C050DF4F68817981DB
:1010B000C050D140AE014E5F5E4FCE0180549F4F75
:1010C0000E94BE08CE5FDE4F88819981AA81BB81D4
:1010D000C250D140CC5ADE4F88839983AA83BB8308
:1010E000C455D140CA5FDE4F88819981AA81BB81F6
:1010F000C650D140C85ADE4F88839983AA83BB83E8
:10110000C855D140C65FDE4F88819981AA81BB81D5
:10111000CA50D140C45ADE4F88839983AA83BB83C7
:10112000CC55D140C05FDE4F68817981C051D1403C
:101130004FE350E0CE018C5E9E4F0E948A0BCE01A1
:101140008C5E9E4F0E94080680E090E0CD5FDD4FF0
:101150000FB6F894DEBF0FBECDBFDF91CF911F91C8
:101160000F91FF90EF90DF90CF90BF90AF909F9046
:101170008F907F906F905F904F9008958F929F9285
:10118000AF92BF92CF92DF92EF92FF920F931F9395
:10119000CF93DF93CDB7DEB7C054D1090FB6F89423
:1011A000DEBF0FBECDBF4B01672B09F46CC020E042
:1011B00030E060E070E0A12CB12C6E01E5E0CE0ED5
:1011C000D11CFE0131967F01FC01E20FF31F20814B
:1011D000211127C0DB011196A80FB91FFE0131961E
:1011E0002D912193EC15FD05D9F76C5F7F4FF5012B
:1011F000EE0FFF1FEE0FFF1FE40FF51F09811A818D
:101200002B813C810083118322833383FA0124855F
:1012100035852F5F3F4F3587248795012F5F3F4FDF
:101220005901FC01E60FF71F2081213021F59B01B8
:101230002F5F3F4FFC01E20FF31FE081EE2399F097
:101240006E5F7F4FDC01A60FB71FF701B9016F5F1B
:101250007F4F2D91219330E08F010E191F09021746
:101260001307ACF301C0B90129813A81FA0137872C
:101270002687118A108A6F5F7F4F9B016815790559
:1012800008F4A2CF02C0A12CB12CFA01B586A48625
:10129000C05CDF4F0FB6F894DEBF0FBECDBFDF914D
:1012A000CF911F910F91FF90EF90DF90CF90BF9063
:1012B000AF909F908F9008954F925F926F927F9220
:1012C0008F929F92AF92BF92CF92DF92EF92FF9256
:1012D0000F931F93CF93DF93CDB7DEB7C255D109DC
:1012E0000FB6F894DEBF0FBECDBF22968FAE229709
:1012F00023969FAE23972496AFAE24972596BFAE34
:1013000025972696CFAE26972796DFAE2797289665
:10131000EFAE28972996FFAE29972A960FAF2A9706
:101320002B961FAF2B972C962FAF2C972D963FAF58
:101330002D972E964FAF2E972F965FAF2F976096D3
:101340006FAF609761967FAF619762968FAF62973C
:1013500063969FAF6397A7960EAD1FADA7972F9685
:10136000CEACDFAC2F9763966EAD7FAD6397C114A3
:10137000D10409F466C07801CE018F5B9F4F5601FE
:10138000AA0CBB1CAA0CBB1CA80EB91EAE014B5F5D
:101390005F4FF7011192DC014D905D906D907D9053
:1013A000CD0149825A826B827C82DE0111963D9189
:1013B0003193A417B507D9F7B5E0EB0EF11C8A15E8
:1013C0009B0539F79601220F331F220F331F2C0D77
:1013D0003D1D6115710509F1D801A20FB31F81E010
:1013E0008C93D9011196A00FB11F2E5F3F4F6C93C4
:1013F00061968EAD9FAD61979A838983DE011196C8
:10140000F801E20FF31F80E090E02F5F3F4F4D9116
:101410004193019686179707C0F3A996EEADFFADED
:10142000A9973183208313C081E0F8018083618311
:1014300061968EAD9FAD61979A83898322E030E0FB
:10144000DDCF6115710581F720E030E0E6CFCE5A9F
:10145000DF4F0FB6F894DEBF0FBECDBFDF91CF9147
:101460001F910F91FF90EF90DF90CF90BF90AF90C2
:101470009F908F907F906F905F904F900895FC01A8
:1014800081E090E030A121A1321711F080E090E0DE
:101490000895FC0121A130E02F5F3F4F2F7130787C
:1014A000332334F421503109206E3F6F2F5F3F4FBB
:1014B000FC0140A150E081E090E02417350711F0D5
:1014C00080E090E008951F93CF93DF93EC01162FF7
:1014D0000E94490A892B81F489A190E0FE01E80F5E
:1014E000F91F108301968F719078992324F4019746
:1014F000806E9F6F019689A3DF91CF911F91089510
:10150000FC0120A181A12817B1F030E0DF01A20F7A
:10151000B31F4C9150E02F5F3F4F2F713078332332
:1015200034F421503109206E3F6F2F5F3F4F20A3CD
:10153000842F952F08958FEF9FEF089588EF809364
:10154000C10086E08093C2001092C50087E68093B8
:10155000C40008950F931F93CF93DF936115710516
:1015600099F08C01EC01060F171F8EE693E00E94A4
:10157000490A892B49F4699170E08EE693E00E9454
:10158000630AC017D10789F7E1ECF0E0808180643D
:101590008083DF91CF911F910F9108958F929F9239
:1015A000AF92BF92CF92DF92EF92FF920F931F9371
:1015B000CF93DF938B01EC01C12CD12C76014B0131
:1015C000A12CB12C0AC08CE493E00E94800A89937C
:1015D0008FEFC81AD80AE80AF80A8CE493E00E9450
:1015E0003F0A892B29F4C814D904EA04FB0458F3F0
:1015F00020E030E00C151D052E053F0510F0C6015A
:1016000002C08FEF9FEFDF91CF911F910F91FF905D
:10161000EF90DF90CF90BF90AF909F908F90089504
:101620001F920F920FB60F9211242F933F934F9357
:101630005F936F937F938F939F93AF93BF93CF935A
:10164000EF93FF93C091C6008CE493E00E94490A97
:10165000892B31F46C2F70E08CE493E00E94630AD4
:10166000FF91EF91CF91BF91AF919F918F917F911A
:101670006F915F914F913F912F910F900FBE0F90FF
:101680001F9018951F920F920FB60F9211242F934F
:101690003F934F935F936F937F938F939F93AF93FA
:1016A000BF93EF93FF938EE693E00E943F0A892B4E
:1016B00039F48EE693E00E94800A8093C60005C04C
:1016C000E1ECF0E080818F7B8083FF91EF91BF910F
:1016D000AF919F918F917F916F915F914F913F91CA
:1016E0002F910F900FBE0F901F901895AA1BBB1B38
:1016F00051E107C0AA1FBB1FA617B70710F0A61B12
:10170000B70B881F991F5A95A9F780959095BC0132
:10171000CD010895FB01DC014150504048F001909B
:101720000D920020C9F701C01D9241505040E0F7D2
:101730000895A0E0B0E0EFE9FBE00C94800EAE016C
:101740004B5F5F4FFA0161917191AF0180919203FC
:10175000909193030E94DF0BE2E00C949C0EAEE0AC
:10176000B0E0E5EBFBE00C947E0E0D891E898F89BD
:10177000988D26E02C831A83098397FF02C080E0AE
:1017800090E801979E838D83AE01455E5F4F698D22
:101790007A8DCE0101960E94DF0B4D815E8157FD4F
:1017A0000AC02F813885421753070CF49A01F801BB
:1017B000E20FF31F10822E96E4E00C949A0EABE039
:1017C000B0E0E5EEFBE00C94700E6C017B018A0149
:1017D000FC0117821682838181FFCCC1CE01019664
:1017E0003C01F6019381F70193FD859193FF81916F
:1017F0007F01882309F4BAC1853239F493FD8591BC
:1018000093FF81917F01853229F4B60190E00E9417
:10181000D60DE7CF912C212C312CFFE1F315D8F018
:101820008B3279F038F4803279F08332A1F4232DB1
:1018300020611DC08D3261F0803369F4232D216059
:1018400016C0832D8260382EE32DE4603E2E2AC020
:10185000F32DF8601DC037FC2DC020ED280F2A3075
:1018600040F08E32B9F436FC81C1232D2064322E33
:1018700019C036FE06C08AE0989E200D1124922ED3
:1018800011C0EAE02E9E200D1124222EF32DF062CD
:101890003F2E08C08C3621F4832D8068382E02C07C
:1018A000883641F4F70193FD859193FF81917F0183
:1018B0008111B3CF982F9F7D9554933028F40C5FFE
:1018C0001F4F9FE399830DC0833631F0833771F04A
:1018D000833509F059C021C0F801808189830E5FEA
:1018E0001F4F88248394912C530113C02801F2E0E8
:1018F0004F0E511CF801A080B18036FE03C0692D47
:1019000070E002C06FEF7FEFC5010E94CB0D4C016C
:101910008201F32DFF773F2E16C0280122E0420EF0
:10192000511CF801A080B18036FE03C0692D70E023
:1019300002C06FEF7FEFC5010E94C00D4C01F32D77
:10194000F0683F2E820133FC1BC0822D90E0881688
:101950009906B0F4B60180E290E00E94D60D2A9478
:10196000F4CFF50137FC859137FE81915F01B60117
:1019700090E00E94D60D21102A9421E0821A91084D
:101980008114910471F7E8C0843611F0893641F56D
:10199000F80137FE07C060817181828193810C5FFD
:1019A0001F4F08C060817181072E000C880B990BB6
:1019B0000E5F1F4FF32DFF763F2E97FF09C09095C6
:1019C0008095709561957F4F8F4F9F4FF0683F2EA8
:1019D0002AE030E0A3010E94120E882E861845C02E
:1019E000853731F4232D2F7EB22E2AE030E025C03A
:1019F000932D997FB92E8F36C1F018F4883579F080
:101A0000B5C0803719F0883721F0B0C0E92FE06108
:101A1000BE2EB4FE0DC0FB2DF460BF2E09C034FEF7
:101A20000AC0292F2660B22E06C028E030E005C08B
:101A300020E130E002C020E132E0F801B7FE07C04B
:101A400060817181828193810C5F1F4F06C060812C
:101A5000718180E090E00E5F1F4FA3010E94120E83
:101A6000882E8618FB2DFF773F2E36FE0DC0232DC6
:101A70002E7FA22E891458F434FE0BC032FC09C00C
:101A8000832D8E7EA82E05C0B82CA32C03C0B82CA5
:101A900001C0B92CA4FE0FC0FE01E80DF11D80812C
:101AA000803321F49A2D997EA92E09C0A2FE06C08A
:101AB000B394B39404C08A2D867809F0B394A3FC40
:101AC00011C0A0FE06C0B21488F4280C922C9B18FA
:101AD0000EC0B21460F4B60180E290E00E94D60D10
:101AE000B394F7CFB21418F42B1802C0982C212C01
:101AF000A4FE10C0B60180E390E00E94D60DA2FEC5
:101B000017C0A1FC03C088E790E002C088E590E020
:101B1000B6010CC08A2D867859F0A1FE02C08BE276
:101B200001C080E2A7FC8DE2B60190E00E94D60DD4
:101B3000891438F4B60180E390E00E94D60D9A949F
:101B4000F7CF8A94F301E80DF11D8081B60190E092
:101B50000E94D60D8110F5CF222009F442CEB601A5
:101B600080E290E00E94D60D2A94F6CFF60186819D
:101B7000978102C08FEF9FEF2B96E2E10C948C0EC1
:101B8000FC010590615070400110D8F78095909548
:101B90008E0F9F1F0895FC0161507040019001104D
:101BA000D8F7809590958E0F9F1F08950F931F93E0
:101BB000CF93DF93FB01238121FD03C08FEF9FEFC4
:101BC0002CC022FF16C046815781248135814217DF
:101BD000530744F4A081B1819D012F5F3F4F3183B2
:101BE00020838C93268137812F5F3F4F3783268355
:101BF00014C08B01EC01FB010084F185E02D0995F7
:101C0000892BE1F6D80116968D919C911797019634
:101C100017969C938E931697CE01DF91CF911F91CB
:101C20000F910895FA01AA27283051F1203181F14E
:101C3000E8946F936E7F6E5F7F4F8F4F9F4FAF4FD4
:101C4000B1E03ED0B4E03CD0670F781F891F9A1FE7
:101C5000A11D680F791F8A1F911DA11D6A0F711D9B
:101C6000811D911DA11D20D009F468943F912AE0A7
:101C7000269F11243019305D3193DEF6CF0108958F
:101C8000462F4770405D4193B3E00FD0C9F7F6CFC0
:101C9000462F4F70405D4A3318F0495D31FD405288
:101CA000419302D0A9F7EACFB4E0A695979587951E
:101CB00077956795BA95C9F70097610571050895FD
:101CC0009B01AC010A2E06945795479537952795A9
:101CD000BA95C9F7620F731F841F951FA01D089541
:101CE0002F923F924F925F926F927F928F929F922C
:101CF000AF92BF92CF92DF92EF92FF920F931F931A
:101D0000CF93DF93CDB7DEB7CA1BDB0B0FB6F894CA
:101D1000DEBF0FBECDBF09942A88398848885F840A
:101D20006E847D848C849B84AA84B984C884DF807B
:101D3000EE80FD800C811B81AA81B981CE0FD11D5F
:101D40000FB6F894DEBF0FBECDBFED010895F89435
:021D5000FFCFC3
:101D520065727220696E206765745F6672616D6577
:101D62003A2025640A000000891112239B3224467E
:101D7200AD573665BF74488CC19D5AAFD3BE6CCA8D
:101D8200E5DB7EE9F7F88110080193331A22A556A4
:101D92002C47B7753E64C99C408DDBBF52AEEDDA6D
:101DA20064CBFFF976E802218B3010029913266783
:101DB200AF763444BD554AADC3BC588ED19F6EEB4D
:101DC200E7FA7CC8F5D983310A2091121803A77764
:101DD2002E66B5543C45CBBD42ACD99E508FEFFB2D
:101DE20066EAFDD874C904428D5316619F702004BF
:101DF200A9153227BB364CCEC5DF5EEDD7FC68880D
:101E0200E1997AABF3BA85520C4397711E60A11423
:101E12002805B3373A26CDDE44CFDFFD56ECE998EC
:101E22006089FBBB72AA06638F7214409D51222502
:101E3200AB343006B9174EEFC7FE5CCCD5DD6AA9CC
:101E4200E3B8788AF19B87730E6295501C41A335E3
:101E52002A24B1163807CFFF46EEDDDC54CDEBB9AC
:101E620062A8F99A708B088481951AA793B62CC23E
:101E7200A5D33EE1B7F04008C919522BDB3A644EB4
:101E8200ED5F766DFF7C899400859BB712A6ADD27B
:101E920024C3BFF136E0C1184809D33B5A2AE55E94
:101EA2006C4FF77D7E6C0AA583B4188691972EE35A
:101EB200A7F23CC0B5D14229CB38500AD91B666F74
:101EC200EF7E744CFD5D8BB502A499961087AFF33B
:101ED20026E2BDD034C1C3394A28D11A580BE77F54
:101EE2006E6EF55C7C4D0CC685D71EE597F4288096
:101EF200A1913AA3B3B2444ACD5B5669DF78600C34
:101F0200E91D722FFB3E8DD604C79FF516E4A990FA
:101F12002081BBB332A2C55A4C4BD7795E68E11C13
:101F2200680DF33F7A2E0EE787F61CC495D52AA1D9
:101F3200A3B03882B193466BCF7A5448DD59622DF3
:101F4200EB3C700EF91F8FF706E69DD414C5ABB1BA
:101F520022A0B9923083C77B4E6AD5585C49E33DD3
:101F62006A2CF11E780F252E32662E252E32662E11
:101F7200252E326600776F72642077617220696E57
:101F8200206E657720776F726C6420696F206578A8
:021F920000004D
:00000001FF
